:020000040000FA
:10000000956A8C6A8A6AF19EFF0E936E0F0EC16E1E
:100010008D6A966A060E846E226A8150010AD8B4EF
:1000200028EF00F0030AD8B43EEF00F0060AD8B477
:1000300035EF00F00C0AD8B44AEF00F0180AD8B433
:1000400053EF00F0300AD8B464EF00F00DEF00F089
:1000500098EC00F08336D8A028EF00F098EC00F080
:100060008332D8A02EEF00F01200800E836E98EC41
:1000700000F08332D8A037EF00F0120022481200BF
:100080000700226E75EC00F098EC00F098EC00F0A0
:100090003EEF00F0AA0E836E98EC00F0550E836ED2
:1000A00098EC00F01200180E836E98EC00F0240E0D
:1000B000836E98EC00F0420E836E98EC00F0810E97
:1000C000836E98EC00F01200810E836E98EC00F0C5
:1000D000420E836E98EC00F0240E836E98EC00F0D4
:1000E000180E836E98EC00F0120022500F0B306E49
:1000F00022380F0B316E1200FA0E246E0000000041
:10010000242E7EEF00F01200010EFA6E23502324FD
:10011000F9263F0C060C5B0C4F0C660C6D0C7D0C2D
:10012000070C7F0C6F0C770C7C0C390C5E0C710C7F
:10013000FA0E206EFA0E216E000000000000000092
:10014000212E9CEF00F0836A040E846E30C023F0F1
:1001500084EC00F0836E7CEC00F0836A020E846E07
:1001600031C023F084EC00F0836E202E9AEF00F073
:0201700012007B
:020000040030CA
:04000000000C1F1EB3
:02000500038175
:060008000FC00FE00F40E5
:00000001FF
